:1000000002780030B402D25A021CB1758C10D26B47
:10001000021A2630B502D25B021D1E32FFFFFFFF1F
:10002000FFFFFF32FFFF0200314CF53139535645D7
:10003000208520F0E4787FF6D8FD85F0203001039C
:1000400012374490F40F7403F090F41FF030011A4B
:1000500012210F50726F6772616D20636865636B68
:1000600073756D202D2D2D2D2000E4FBFF900000D9
:10007000E4932BFBE43FFFA3744CB583F374F3B517
:1000800082EEE4932B7006A3E4932F600E90074258
:10009000120EF412271E7590FD80FE122710749622
:1000A000120EF97583F01237F47583F41237F49059
:1000B000F4187888D2F1D2F012380D745A1228E769
:1000C000C374CD94F5F5047463944CF5051228E7D8
:1000D000E5041228E7904CF50505E4931228E7A300
:1000E000D504F7D505F4E493A31228E7E493A3120B
:1000F00028E774A13002027461FE7C007940122866
:10010000E7120130122936F709500AF8EEC4440FFD
:1001100068D36001C3EC92E303FC0EEE30E2DF90A3
:100120000128EC93F57780110307000B0000000F06
:100130007B127A00DAFEDBFC2220010302026C1241
:10014000210F536C61766520636F6D6D756E696309
:100150006174696F6E202D2000E577600302023222
:1001600012210F4552524F5220007840E61245C3EB
:1001700008E61245C308E61245C312210F0D0A0016
:1001800012018E900758120EF47590FE80FE7C01CD
:10019000794012210F202020536C617665202300C6
:1001A000EC24301245EAE76057F5F012210F2020C9
:1001B000204570726F6D202D2000A2F012021E12D9
:1001C000210F20202052616D202D2000A2F112026B
:1001D0001E12210F202020492F4F202D2000A2F297
:1001E00012021E12210F20202050726F6772616D63
:1001F000206C6F6164202D2000A2F312021E801279
:1002000012210F2020204E6F20726573706F6E7365
:10021000650012272B0C09BC04012202019240093F
:1002200012210F42414420002212210F474F4F4418
:10023000002212210F474F4F440D0A2020204E75F7
:100240006D626572206F6620706F727473206465D2
:10025000746563746564203D2000AD770D7A00C23B
:100260002112274E12272B7496120EF9E57790E48F
:10027000F5F030010312018E30030302031775A05D
:10028000E579009064007D017C407F007B00E49371
:10029000F3120333A309B9000205A0DCF1DDEF7509
:1002A000A0E679009065007C00E493F3120333A389
:1002B00009DCF630011A12210F436F6E6669672060
:1002C000636865636B73756D20202D2D2D2D2000C7
:1002D0009067FEE4932B7030A3E4932F702A90E58F
:1002E00000E0B4012390E501E0B4231C90E502E0B6
:0302F000B4011541
:1002F30090E503E0B4040E122710900817120EF4D1
:100303001208DB804212271E7590FF900700120E21
:10031300F41208C0120543400C9006A8120EF41202
:1003230008C002027E9006D4120EF41208C080DBCD
:100333002BFBE43FFF22012301040005100F2B00D8
:100343001012000000000090E504E0A2E092389053
:10035300E505E090E4FEF0A3F090E506E090E4FC10
:10036300F0A3F090E507E0F57790E508E090E4F37B
:10037300F090E509E090E4FAF0A3F090E50AE0904C
:10038300E4F8F0A3F090E50BE0F55F90E50CE0F501
:100393007690E50DE090E4F6F02001030203C0122D
:1003A300210F2020204D617820706F7274203D2032
:1003B30000E5772401FDE43400FA12274E90E4E7C8
:1003C3007406F030011312210F0D0A496E69746926
:1003D300616C697A696E672000120DF812378653D3
:1003E30089F0438901D28CD2A9D2AF1204551204E9
:1003F3007D1238461204F6D26874FFF570F571F574
:1004030072F57390E4E07400F0A3F0902BC4122B08
:10041300B5122DE4D21690E4EF7479F090E4EE1265
:100423001B953002030208E4120E62121DDD124115
:100433005BB3921B120EE030011512210F0D0A530C
:1004430074617274696E67206D61696E0D0A0002D2
:100453000F58C2A8D2B3D21F755160755060E55FC3
:100463005407B40508C2AA1204CAC2B222B40406CD
:10047300C2AA124C78221204A422C2AAC225755A17
:1004830040755940E55FC45407B405041204CA22F9
:10049300B40403C2AA22B401041204B9221204CA86
:1004A300227525087560AA755061755160D288D28E
:1004B300A8C289D2B222752608D2BAD28AD2AAC2D7
:1004C3008BD2B31226C622E55FC4540FB40204C212
:1004D300F0800CB40304D2F08005B40502D2F078A6
:1004E30066C2F190F40012380D90F41012380D1218
:1004F3000D5722227C07900523E49312052AA3DCDF
:10050300F8E57675F010A42400F582E5F03468F57B
:10051300837C10E49312052AA3DCF8E412052A2253
:10052300637181703F0B7475A0F57909C0E0E33006
:10053300E2FC5301F8430103D0E0F37900D9FE2232
:1005430030012812210F52656C6F6164696E672058
:100553004E5672616D20746F20666163746F727999
:100563002064656661756C740D0A009006EA120ECC
:10057300F41208C0900716120EF474C0120F05127D
:10058300084E7B007F0075A0E779009003397C005B
:10059300E4BC40005021BC3000400474108018BCFF
:1005A300200040047401800FBC10004004740280DA
:1005B3000693BC0702E577F3120333A3090CBC00CF
:1005C300CF90640012063850012290E7007C00743B
:1005D30012F0120333A3DCF79065001206385001C2
:0105E30022F5
:1005E40090E7007C40E4F0A3DCFB7E08906600BE4C
:1005F400010E75A0E7793EC3E49BF309C3E49FF3BE
:1006040075A0E7790012EF805002D322DEE17B016E
:100614007E40906800C082C083C006120660D00687
:10062400D083D08275A0E7790012EF805002D322E4
:10063400DEE3C3227C0075A0E77900EC2582F58215
:10064400EC29F9C004C082C083121A14D083D0826A
:10065400D0044007EC2440FC70DCC322780490E70B
:1006640000D2217C00EC242B83F0BC031CBB0006CD
:100674007D007A0180048B057A00C000C006122731
:100684004ED006D0007C068002A30CBC10D70BD839
:10069400D2C2212243505520202020202020202077
:1006A4002020202080526573657420737563636510
:1006B400737366756C2020202000C048697420651F
:1006C4006E74657220746F2070726F636565640068
:1006D400805265736574206661696C6564202020AE
:1006E40020202020200080436F6E66696775726148
:1006F40074696F6E207265736574200080436F6E39
:1007040066696775726174696F6E20626164202026
:100714002000C02020202020202020202020202055
:100724002020202020202000802020202020202085
:100734002020202020202020202020202000C05005
:10074400726F6772616D20636F7272757074656425
:1007540020202000C0536C617665206C696E6B208C
:1007640062616420202020202000C05374617475CD
:10077400731D206E6F726D616C202020202020007C
:10078400C05374617475731D206E6F20637075207F
:10079400706F77657200C0456E746572A573656C81
:1007A400656374209E9FA56974656D0080536176AE
:1007B4006520636F6E66696775726174696F6E2018
:1007C4002000C0456E7465722063686F6963659E1E
:1007D4009F20596573202000CF59657300CF4E6F59
:1007E4002000805363616E206D6F6465202020209B
:1007F40020202020202020004E616D6500203D2017
:1008040000204368616E676520592F4E2F4553437E
:100814003F200091964F4B004F6E204F6666C053A9
:1008240074617475731D206E6F742073656C6563D9
:1008340074656400C05374617475731D20766964B3
:10084400656F206F66662020200090086675A0EF13
:100854007980E493F3A3097408B583F674C0B58270
:10086400F122C2AFC083C08290555574AAF0902A79
:10087400AA7455F090555574A0F0D082D083C083EB
:10088400C082C0017C40E3F0DC02800409A380F64E
:10089400C200F8E4936820000530E7F7D20020E7AF
:1008A400F2D001D082D0837C40E493F8E3A309B56D
:1008B4000006DCF5C3D2AF22D3D2AF229006BE121B
:1008C4000EF41208D2121C1E50FBB407F822121C9C
:0108D4001E05
:1008D50040FB1208DB2278007900D9FED8FC229073
:1008E500F0007C07786675F00112380D5382F8E543
:1008F500822408F582BC040390F400DCEC90F41823
:100905007888D2F112380D53A8FA30011512210F4B
:10091500446961676E6F73746963206D6F64650DFB
:100925000A0090072C120EF490E4F5E00404FC7420
:1009350083120F05900DDA120F0CD20D90071612C7
:100945000EF4900DF4120EF4200D0A74201228E70F
:10095500900DF0800874101228E7900DEC120EF43B
:1009650090E4F5E0040303145403F5487549007554
:100975004A007549007590FCD2EC200D05120A70ED
:1009850080031209D8C2EC120BE0E5496548054918
:100995006014743045491228E77C0679401228F81E
:1009A500F709DCF980E1054AE54AB46403754A00B4
:1009B50074C0120F057A00AD4AD21ED20512274E19
:1009C500C2050547E547B46408D20C90F8007408E1
:1009D500F0809FD202B2027B0375464020020812C6
:1009E5000D3A120BD28003120D487C047AFB800964
:1009F5007546407C087AFE05462002036302FFEA3D
:100A0500BB0406F5C0E5C0800E500844C3F5B0E54B
:100A1500B08004F5C8E5C86A8A003002036300FFA8
:100A250055006004A84646F6E5D8540F60024243D7
:100A3500E590543C643C600242447E0475A0F07825
:100A450019120BC3E824F8F8DEF775A0F478111233
:100A55000BC3EA23FA120CECDCA50B120D70120B7A
:100A6500B2BB068F300201220209DAC202120D481A
:100A7500120BB27C047AFB7B03E4120BD280067C5A
:100A8500087AFE79FCEABB0408F5C0E5C0A8C88071
:100A95001B5013F5B0E5B044C37F00120C79BF01BC
:100AA50001F442408022F5C8A8C8E5C07F0049127C
:100AB5000C79C849120C79C8BF0106F449C8F44934
:100AC500C8694241E8694242EA23FAEC30E007E9A5
:100AD5002323F9120CECDCAD0BBB06A3E5D8F454CB
:100AE5000F6002F5437C0490F01B785AE8F023F878
:100AF500E58224F8F582DCF4C2EE90F403E8F01206
:100B05000D66120BB27C04785A90F019E030E00FB4
:100B150005820582E015821582B50003C38001D3E5
:100B2500E54533F545E58224F8F582E823F8DCDC74
:100B3500E545C333F54590F411E030E0090582053C
:100B450082E065006003434501D2EEE590543C64C4
:100B55003CF544A202920ED202D2EE120D70E5903F
:100B6500F4543C643C4244120BB290F411E020E78B
:100B75000BC2EE120D66E030E7028003434402C269
:100B850002120D48120BB2C2B2120D66A20E9202EB
:100B9500783A123D9590F401E030E00A058205822D
:100BA500E0B43A028003434310120BB222E590549D
:100BB50003B40307C2EC7590FC8002059022E25451
:010BC500F13E
:100BC600B40100B3E54572E433F54522E4F540F59A
:100BD60041F542F544F543F54522E5415542FD9080
:100BE6000C0C7C045403B40313E493A3FE7F581245
:100BF6000CC7D20FE493524152428001A3A3ED03E6
:100C060003FDDCE0800802FC01F303CF043F900DF6
:100C1600B27C14E5400303540FB40F0D7E007F58D9
:100C2600D20F900DBA7C118013BC1004E5418005EB
:100C3600BC0802E54213FD500D120C85120CC712BA
:100C46000CDCD20F8002A3A3EDDCDE300F05120C04
:100C5600DCC20FE5436006120C8E120CDCE5446024
:100C66000703120CB2120CDCE5456006120CB61234
:100C76000CDC2275F0083340010FD5F0F93322E47D
:100C860093A3FEE493A3FF22FD30E4077E007F5387
:100C9600120CC7ED7F42F5F0A2F092E1A2F192E0CC
:100CA600A2F292E3A2F392E27E0180087F448002E0
:100CB6007F507E00135005FD120CC7ED0EBE05F4E5
:100CC60022E5496006BE000122232324C32E120F0B
:100CD60005EF120EF922D20F79C0E4D9FEC9120C23
:100CE600ECC9D5E0F622120D1E4004C2068016207D
:100CF6000613D206100C0F754700B40702B20D7525
:100D0600810702094122C083C08290F800740CF06A
:100D1600D082D08375470022C006C002C001C00041
:100D2600C083C082121C1ED082D083D000D001D0D6
:100D360002D0062275B0C3E4F5C0F5C8D2EE120D96
:100D4600702275B0FF74FFF5C0F5C8C2EE120D70C3
:100D560022D2EEB15DC2EE79007A40D9FEDAFC22EB
:100D660074127900D9FED5E0FB227C0875A0F078D4
:100D760002BC040775A0F47802800ABC0302802531
:100D8600BC010280207402F2200204747080027496
:100D960060F27445F2120D6618E230E0070808E2C8
:100DA600181880F508E82408F8DCC6220037003950
:100DB600003800410241023901410139034103393A
:100DC6000441043902380237013801370338033742
:100DD6000438043743313233343536373839303115
:100DE600323334353600804F5000804C4200C020EC
:100DF600300012208790E5147E04120E5390E524ED
:100E06007E14120E5390E6047E24E578603790E552
:100E160030E0FA8578F0A42404C39578F5827583CA
:100E2600E67C0C7905EE1228E70EE578B501005050
:100E360005E07A01800274121228E7E5822AF5821B
:100E460009DCE28003120E53E41228E7227C0CEE42
:100E56001228E70EE0A31228E7DCF422E578B402B4
:100E660000402E7C01BC0400C00450098C7474162A
:100E7600123B1880147401122946ECC412294674D8
:100E8600EF1229467416122946E578D0040CB504EB
:100E9600D422C0E0C082758205E4D5E0FDD582F992
:100EA600D082D0E02290F8007430F07406F0740C12
:010EB600F04B
:100EB7002290F800740DF02290F800740CF022755F
:100EC700A0F87900F30975A0F87901E493A3600805
:100ED700B45C02748CF380F32220771090076E20A5
:100EE7001B03900784120EF4A21B921C22E493A307
:100EF70080CD75A0F87901B45C02748CF32275A0DB
:100F0700F87900F32275A0F87901E493B45C0274D0
:100F17008CF3A3DCF5227480120F05E576120F40DF
:100F27007420120EF97A00AD760DBD00047A017DAA
:100F370000D20512274EC20522120F497C10120F4C
:100F47000C2275F010A42400F582E5F03468F583CF
:100F570022306B03121A39305708C257203903124F
:100F67002BAAE55F540FB40416D55B26755B10E515
:100F7700537003124984E55C70181249D6801340F8
:100F87000812211F1221458009E55F6412600312D0
:100F97002145205E0C20700C207109206F06020F7E
:100FA700F30212E77D04E55C6015207209D27290A6
:100FB700E4CFE4F0803390E4CFE0B40200402AC2EB
:100FC70072E55FC4540FB4012030251574F5D27F44
:100FD7001225F8EF6009122666400464FA6002DD04
:100FE700DE75260885595AD26E121DDD301950124A
:100FF7002936504BF8121001804530E731B4800B89
:10100700D268300139747E1245EA2230E60B53006C
:101017000F12151754F048F02230E505A2E0921B95
:101027002230E41AD2201214F8E8540FF022758304
:10103700E4E575C4540F44D0F582E8F0D27522E593
:1010470076B40400501574382574F82404F9E6546E
:10105700137005E7541360030213E9300402801E7E
:1010670030272090E4E0E0F8A3E0C868601375A09B
:10107700E8E2F556D20408B8C0027800E8F0021298
:101087003BC227E550B551028076E55F540FB404A3
:1010970000501BA851E6B4F706D211D2148007B44A
:1010A700F80CC211D214055153516F0212E71222E4
:1010B7000430011930041674201245EA745512459C
:1010C700EAE5561245C37005E5571245C3102302DA
:1010D700802ED23912371B1245C3E550B551028015
:1010E700F91215A212371B1245C30227B0E550B5F6
:1010F700510280F91215A21237201245C30228ACFB
:10110700207C03021202E553600302123B300410F5
:10111700AE56BE2E0EC210C27CC2507C2D12186273
:101127000211FD201042BE79217C22121862C250A2
:10113700D21090E4C77401F090E4C8E0122F087C45
:10114700107420F0A3DCFC0211FDBE6ED390E4C83E
:10115700E004B5770280034001E4F07C2D121862A9
:10116700121823C2040212327445A879B8550274C2
:1011770051B5061490E4C7E0B40102807914F01267
:101187002F087420F002123BBE4718122F58C210C6
:1011970090E4C8E0B57603120F1D90E4C7E0240A77
:0111A700FC4B
:1011A80080BABE4805D25002123BBEC805C25002E2
:1011B800123BBE8000507CBE2E004039BE48005015
:1011C8000E902B48305003902B62EE93FE8011BE98
:1011D8007B005021BE6100401CEE30500324E0FE2D
:1011E80090E4C7E06411600D122F08EEF090E4C798
:1011F800E004F0803EC2040212E72039363004339E
:10120800E556B44A04D267802AB4CA1230671BE58F
:101218005F5407B40504D2538019D2768015B42DD3
:1012280009305306D276C2538009E4F52CF57AC208
:101238005EC25330190730045EC2048037E553702C
:101248002C30045330181AE5566007B42D13E47592
:10125800572DE557B419004008123B18C204021272
:10126800E7123915E553606B7555B0C20475A0E4F3
:10127800A855E2F8301923122905E556B42D04E4DF
:1012880075572D7001F41228E7B4FF47E557A218E7
:1012980092E61228E7803C0212E712415B403020B8
:1012A8001818E5795407B4040875F0FF1245F5805D
:1012B800124007E5741238508009E574124093E82B
:1012C8001240BB500A0554E554B40A13755400057E
:1012D800551553307609E5537005C276021522304C
:1012E80073028026E559B55A02801F12243B30014B
:1012F8001930731674751245EA90E4BDE01245C3BF
:10130800A3E01245C3A3E01245C3E55C7021307326
:1013180013301905123BEE8003123B2D307B077505
:101328005C00C2738062E55C605E755EB8C273750E
:10133800A0E4A95EE3F830193212290590F41A7472
:1013480015F07582187407F090E4B8E0A31228E746
:10135800D55CF890F419E030E3FC30E2F990F41A27
:101368007415F07582187403F0807612415B406D35
:10137800201833E579C45407B4041F88F009E3F84A
:101388001246124006755C000213E9055DE55DB47E
:10139800104F755D00755C0080474007E574123892
:1013A80097802EB40126E574903911935529602D44
:1013B8008000E5749040B793FAE5C0035A6022E5CF
:1013C80074D2E2124093E81240BB8005E5741238EB
:1013D80097500A055DE55DB41007755D00055E155B
:1013E8005C123C59106C1810526810137A102015B2
:1013F800105155101267106E761075060214ED0222
:10140800149B0214AD1214F8F8E55F5407B40407EE
:10141800E8124CC50214ED4025C000780E123D803C
:10142800D000E8A2E092F2A2E192F0A2E292F3A246
:10143800E392F153F00FA8F0123D800214ED74ED21
:1014480012148CD26C0214ED74F012148CD2520265
:1014580014ED121517540312148C0214ED74F112C2
:10146800148CD2130214EDE57612148C0214ED30AC
:10147800257385595A74F41225F8EF6068122666A8
:10148800C27F80617D03FB12258C1215E35003EBAC
:02149800DDF580
:10149A00221214F85407303905A21BB392E712142A
:1014AA008C80407583E4E575C4540F44D0F582E816
:1014BA00E0F8E55F5407F9E579540FB40402802394
:1014CA004012B80E0302140D203912B90515E8129C
:1014DA003D80800FB8ED0302140DB9ED06E8121431
:1014EA008C8000C275205E03020F5802152A75838C
:1014FA00E5E575C4540F4410F582E022C3E575543E
:10150A00C07009E575C45403B50401D3227583E696
:10151A00E5764400F582E022757E00D25E757C0095
:10152A00E57C206A06B420090215F1B420030215ED
:10153A00F1C3E55024109551540FF8E55F5407B4F0
:10154A00041CB8020040601215A2FE1215A230E770
:10155A000ACE20E70653067F6E604F0215FA402135
:10156A00B8030040421215A2FE1215A230E7ECCED3
:10157A0020E7E853067F6E70E21215A2B47FDC8082
:10158A0029B8030040211215A2FE1215A2B4F0CB0D
:10159A001215A26E70C58012A851E612370C1245B8
:1015AA00C3055153516F22020F58EE12220730041D
:1015BA00AAC204AE567C009017B4E493609DB506A7
:1015CA00028004A30C80F39017D2EC230493C0E0AA
:1015DA00EC2393C0E0220215FDC378007908102697
:1015EA0005D8FBD9F9D322E52C547F7003021626BD
:1015FA00855051757A00752C00C25E0212E70217F7
:10160A001D0218940218A920602B20614B20626EDB
:10161A002063EB2064252065E82066E812167040F6
:10162A0034F57EE577B57E00402B857E76C238C2DA
:10163A0070D26F802090E4FC021720E57F70B1E53C
:10164A007EB4800050AAC082C08390E4F3F0D083B5
:10165A00D0821226A902123212167040936091F5B6
:10166A0077121DDD80EF857FF0E5F0B40200500CA3
:10167A00E57E20F005600514C32260FBD322E57ED7
:10168A00B40A0050666064FAF9121517BA040474B1
:10169A0044802BBA0504745580244011540FB404B5
:1016AA0000506DCA24FBB404137405800FC4540F90
:1016BA00A87953000FB8040040027401C44AF579AE
:1016CA00201806121517E579F020183120191EB9CD
:1016DA000500403CD2F0B90702C2F07583F0E57408
:1016EA00C403F5827866C2F112380D8023E575C409
:1016FA00540F4440122946E01229468013E9243047
:10170A00F97A6D1223B889021223B87A471223B8DC
:10171A0002123290E4F8E57F4410F0A3F0A3E57ECC
:10172A00F0A3F0021232D238021232C23802123256
:10173A00D270C2388009D27180F8A201B392010234
:10174A001232D260800ED265800AD2668006D261D9
:10175A008002D2620215271237441226881226C640
:10176A00120D57C2381220C180D5D26380E6D26AE0
:10177A00E57E75F00AA42C500205F0F57E85F07F0F
:02178A00E52C4C
:10178C00547F701D057AE57AB4020AE577B46300DC
:10179C00500F02162650FBE577B4090050030216D1
:1017AC0026021527D26480AA3031323334353637CD
:1017BC003839477378746B3B3A43706D72766E614F
:1017CC006977752E0C0017781778177817781778B3
:1017DC001778177817781778177816111730173578
:1017EC00174C190A173A174017441758175C17610A
:1017FC00177418CE17B018BB17501754188C180E36
:10180C0015FAD27C90E4C8E576F0C2507A481223DF
:10181C00B812182302123290E4C8E0FF9007FC12B1
:10182C0023D3D221EF2401FDE43400FA90E4CB124F
:10183C00274EE4F090E4CB1223D3C221900801127E
:10184C0023D3EF120F497C101223E3EF122E4D908D
:10185C0008051223D32290E4E0E0F875A0E8744563
:10186C00AB79BB55027451F2D2E708B8C0027800CC
:10187C00F2C2E708B8C0027800DCECE8F0D227220C
:10188C00305602D27B021232E57F700EE57EB40236
:10189C0000400790E530F00212320215FAE57F7035
:1018AC000BE57E90E4F6540FF00212320215FA7E2C
:1018BC0000903752EE936007FA1223B80E80F202B2
:1018CC0012321218D4021232E579540FB4040050BB
:1018DC001120180F201921E574D2E2124093E41262
:1018EC0040BB22E57412409374EF1240BBE57412B6
:1018FC00409374311240BB227431122946221219C2
:10190C0010021749121919121977500022E5787034
:10191C000302196D7B00EB124093C21974EF124055
:10192C00BBEB12409374151240BB0BBB0402800737
:10193C00E578B503E1802AE57824FC6024FB757515
:10194C0040D219D2187401122946E575122946D2D3
:10195C00237415122946E5752410F575120E98DBC3
:10196C00E4203906121E8E121DDD2290E4FEE0905A
:10197C00E505F090E4FCE090E506F0E57790E507EE
:10198C00F090E4F3E090E508F090E4FAE090E509DB
:10199C00F090E4F8E090E50AF0E55F90E50BF0904C
:1019AC00E4F6E090E50DF012084E7B007F007C40E1
:1019BC0090E500E493120333A3DCF875A0E77900FB
:1019CC0090E6007C00E493F3120333A309DCF69059
:1019DC00640075A0E57900121A145001229065007C
:1019EC0012063850012290E7007C40E4F0A3DCFBA7
:1019FC0090E73EC3E49BF0A3C3E49FF09067C075EF
:101A0C00A0E77900121A14221221C1C2A912EF8088
:101A1C0092F01221A5D2A9A2F022202B06107E034F
:101A2C00752508203306107D0375260832C26B30ED
:101A3C00790F307708121F0DC277120EE0C2798031
:101A4C001690E4F9121BB6501420770B121EE3D239
:101A5C0077900838120EF490E4F8121BAEE57B3048
:101A6C00E602D25F046002F57B057C90E4CFE004D3
:011A7C00F079
:101A7D0010490385595A123FAAE55F540FB404006B
:101A8D005004A21F8002A2B32016045046800240CB
:101A9D00429216E579540F92F0B404004035A2F04D
:101AAD0020190820181412416F8028740B400674F9
:101ABD000AA21892231229468019E57412409374D4
:101ACD00EF1240BBE574124093740B201602740A9A
:101ADD001240BB201118201A1530381290E4FD1257
:101AED001BB6500AD215D27090E4FC121BAE303FDB
:101AFD001C90E4F7E004F0B402004011C23F12283C
:101B0D0015900822120EF490072C120EF420116A73
:101B1D00201A41203E02801090E4E3E0B41E004004
:101B2D0005122C08800204F0201A292019133018F0
:101B3D000A1214F8A2E7B3921B800612415BB3920E
:101B4D001B201C05301B0D8003201B08303902D2D1
:101B5D0020120EE0121BD99257501F90E4E3E4F0CF
:101B6D00D27990E4EF7479F090E4EE30221A90F887
:101B7D0000740CF0C257C222802690E4EDE014F000
:101B8D00701EA3E014F070187404F015827484F0C4
:101B9D0090E4EFE014F0700890F8007408F0D22291
:101BAD0022E0A3F0A3E0A3F022E02410F05019F8F6
:101BBD004410F0A3A3E0B80002600D14F07009E822
:101BCD0060081415821582F0C322D322121C1E4008
:101BDD0008C20690E4E6E4F022901C719360F214C2
:101BED00FE3006028004D3D20622BE0B02800DBE4B
:101BFD000C028008BE0E028003BE0F1390E4E6E0D7
:101C0D000430E30A2408B4280050DBF080D8F0C378
:101C1D002275A0F47583F4780D791D75820E7A0105
:101C2D00121C5EB40F2975820E7A02121C5E2410EE
:101C3D00B41F1C75821E7A01121C5E2420B42F0F56
:101C4D0075821E7A02121C5E2430B43F02C322D369
:101C5D0022EAF0E25403FEE35403232342060582F5
:101C6D00EAF0EE22000000000000000E0000000867
:101C7D000005020000000000000000010000000946
:101C8D0000060300000000000000000F0000000A25
:101C9D000007040000000000000000100000000D0F
:101CAD00000C0B00202F1E302B0A105A63D279D254
:101CBD007E152532C55203D2E7105A02C2E7C5522E
:101CCD001525C22B32102835752508105A03D274EC
:101CDD00323058FAC2B2C001C55264FA7008D22629
:101CED00C5527930801064FAC552A950A7520953D4
:101CFD00016F8950792DD9FED2B2D00132C552D2A1
:101D0D0058105A0520D007800330D002C258C55252
:101D1D003220372030330C105B49D279D27DD24935
:101D2D00152632C55B03D2E7105B02C2E7C55B1512
:101D3D0026C23332103019752608105B0132305926
:101D4D0022C001A959A75B0953014F8959D001320E
:101D5D00C55BD259105B0520D007800330D002C27D
:011D6D00591C
:101D6E00C55B32E599C298B43F0485769922F59900
:101D7E003099FDC299205E3B105D09A2E0925C7025
:101D8E0015D25D22C0E0E574A25C92E2124093D0BF
:101D9E00E01240BB801DF890E4E2E0C8B40D1518C7
:101DAE00E577B50000400A8876D215C270C238D2E7
:101DBE006FE4F02224D0B40A0050F8C8C0F075F0D9
:101DCE000AA4D0F030D20280EA285001E4F022209A
:101DDE005E1E20511B202018206C152052121070F0
:101DEE001010711CC26FE577B576004003021E1B02
:101DFE00220576E577B576005013757600021E1B28
:101E0E001576E576047006857776021E1B74AA4257
:101E1E00C0D21F124182201A03120F1D1204F71294
:101E2E001F40121E8E301810121FC1120E9830193C
:101E3E0012740C122946800B121FC1C2EC12204BD9
:101E4E00120E98121F78301827201917E575C454F2
:101E5E0003C082C083903911934529F529D083D0D0
:101E6E0082800D7430122946E575C454031229463A
:101E7E00201A03120EE010150122301402D2122283
:101E8E00A976121EA4F575F9A876122181A2F692F2
:101E9E0019A2F7921822203907122087E5787006CA
:101EAE00E9C454F0802EE578B40F03E980268578D6
:101EBE00F090E530E0A414B50100500BC304F5F02A
:101ECE00E995F0257880DA90E530E0F5F0E9845474
:101EDE000FC445F02220180520191C801FE575C47B
:101EEE00540312409374EF1240BBE575C4540312B1
:101EFE00409374021240BB7402122946C2EC222097
:101F0E0019052018028028301905740C1229463044
:101F1E00181FE575C4540312409374EF1240BBE5CD
:101F2E0075C45403124093740C1240BB201902D294
:101F3E00EC2220192030181AE575C4540312409370
:101F4E0074EF122162E575C4540312409374161295
:101F5E002162C2EC2230180A74EF1229467416124E
:101F6E0029467402122946C2EC2220184030192943
:101F7E007409122946122914D268F854706018E8B0
:101F8E00A2E7921B1214F8E8540FF0E8C45407F8B5
:101F9E0012151754F048F08003121517F579D22058
:101FAE0030390A540FB404005002D25122121517C0
:101FBE00F57922E57554C060387401122946E5752D
:101FCE0054F0122946740C122946301823120E981A
:101FDE00120E9874EF122946120E987401122946A9
:101FEE00120E98E575540F122946120E9812204BB8
:101FFE002230183DE575C45403F57444FCF590D2B7
:10200E00ECE575C45403F57412409374EF1240BBA3
:10201E00E575C45403F57412409374011240BBE588
:10202E0075C45403F574124093E575540F1240BBFA
:10203E0022E575C45403F57444FCF590222019066C
:10204E00201803D2EC2230190AC2EC740C12294665
:03205E0030182512
:10206100301908E575C4540312409374EF1240BB54
:10207100301908E575C45403124093740C1240BB27
:10208100201902D2EC22C083C08220390A90E4F6E2
:10209100E06004F578800F75780020390990E4F547
:1020A100E0B577004005D082D0832290E530E0F59D
:1020B100F0E577B4FF04540F80020484F57880E6DC
:1020C10020181020193A903911E5745403934529C9
:1020D100F52922301903122101E5745403124093AA
:1020E10074EF1240BBE574540312409374301240F4
:1020F100BBE5745403124093E575540F1240BB22A3
:102101007430122946E575C4540312294622D0833E
:10211100D082E4931245EAA3E49370F8047390F437
:1021210001E030E01E54E07900600279FF5382F84B
:10213100438203E0B900E7A950F7055053506FD22D
:102141007980DB2290F411E030E0155382F843826C
:1021510003E0A959F7055953594FD249D27980E47F
:1021610022C0E0755400D0E0C0E01240BB500A0527
:1021710054E554B40AF0024111D0E0C37554002271
:1021810075F000203916E5786012F5F090E530E041
:10219100A41475F000B500004002D2F7E954C06004
:1021A10002D2F622C0E0E55F5407B40210D2A8D2F1
:1021B100B2E55FC45407B40104D2AAD2B3D0E0227D
:1021C10030A80C302BFDC2A8C289C2B275250830D7
:1021D100AA0C3033FDC2AAC28BC2B3752608227F76
:1021E100FF30B202DFFB227FFF20B202DFFB227F42
:1021F100FF780830B304DFFBD8F9227FFF20B30258
:10220100DFFB221215A2F8AE5F530607BE04005091
:1022110038E5586003022298B8AA06D25F122688D0
:1022210022B8DF004023B8EF0AD239D223C2387571
:10223100770F22B8F00475580122B8E004755802EE
:1022410022B8E1047558042222E55F5407B404055D
:10225100902A1780204005902A978019C392F09008
:102261002987E893A879B84408B44C052039027449
:102271001BA2F08006E8A2E7C2E79364FF6017643F
:10228100FF30E70975560092E7F557800492E7F5AC
:1022910056D20475580022E558B401028015B402E3
:1022A10004C2F08013B40308D2F09023000222C4C8
:1022B100022385D312225E22E8B4F004755803226A
:1022C100902300E4A393A36015B500F7E49330F0E5
:1022D100022402F557755600D20475580022902346
:1022E10006E893F556A879B8440DB44B0A20390392
:1022F10075561CA2F0921F30F003435680022292C1
:10230100120159020000000000000000000000005E
:102311000000000000004D00004B00000000000024
:10232100000000004E000000000000004F0000000F
:10233100000000001D00000000000000000000007F
:102341000000000000000000000000000000005B31
:05235100000000000087
:10235600000000000000000000005F000000000018
:10236600000000000000000000530058520000006A
:102376005051570059560000000055000D547E90EC
:1023860023A69023ACE55893B500150558E5589358
:1023960070117A0F1223B8742D1224238002D204EE
:1023A600755800221D45E19DC5001477E1F014F033
:1023B600770090E4E0E0F875A0E8EA7C02F208B85D
:1023C600C0027800D2E7DCF5E8F0D227222021040B
:1023D600E4938001E060051223F180F122202104BC
:1023E600E4938001E01223F1DCF322C083C08290E3
:1023F6002AF793FA53027F20E70C305013C2507429
:10240600C8122423800A205007D25074481224236D
:10241600C0041223B8D004D082D083A322C0E09097
:10242600E4E0E0F875A0E8D0E0F208B8C002780071
:10243600E8F0D22722E5592410955A540FF8E55FA3
:10244600C4540FB4040AB80200402A12247C802324
:10245600400CB80500401E1224B540198015B40181
:102466000AB80300400F123C028008B8030040057A
:1024760012251ED27322A85AE6055A535A4F75F0F2
:1024860008A2E7B392F0A2E692E7F404A2E792F577
:1024960090E4BFF0A85AE6055A535A4FA2E692E7CF
:1024A600A2E792F490E4BEF090E4BDE5F0F0227568
:1024B600F008A85AE630E74EF4A2E292F0A2E192C2
:1024C600F2A2E092F10853004FE6FE080853004FCF
:1024D6002690E4BEF0EE6630E701B392F41853009E
:1024E6000F430040E6FE080853004F2690E4BFF075
:1024F600EE6630E701B392F50853004F885A90E430
:10250600BDE5F0F0C3220853004FC3E559986004B7
:10251600E630E7F2885AD32275F000A85AE630E68C
:10252600530853004FA2E592F0A2E492F1A2E19281
:10253600F4A2E392F5A2E092F2A2E292F3E6085345
:10254600004FA2F292E6C392F2A2F492E790E4BEA2
:10255600F0E60853004F885AA2F392E643F008A229
:10256600F592E7F404A2E792F590E4BFF090E4BD9B
:10257600E5F0F0220853004FC3E559986004E630B1
:10258600E6F2885AD322305F6812372A1245C330E2
:1025960033FDC2AAC2B3302BFDC2A8207403122198
:1025A600E8C2B27F3CDFFEC2B4D2B2A2D0B37C098D
:1025B6007E0A7F0030B20BDFFBDEF9D2B48019123F
:1025C60021E01392B41221E8DCF51221E0D2B41214
:1025D60021E81221E01221E8C0E0E55FB41209C249
:1025E6008B752608D2B3D2AAD0E0C289752508D247
:1025F600A82212372F1245C3302BFDC2A8C2B23013
:1026060033FD1221FCC2AAC2A9C2B37F3CDFFEC2BF
:10261600B5D2B3A2D0B37C091221F01392B5122120
:10262600FCDCF51221F0D2B51221FC1221F01221A8
:10263600FC752608C289C28BD2AA752508D2B2D2E9
:01264600A8EB
:10264700D2A92278007908E550B55106D8F9D9F70B
:10265700D322A851E612370C055153516F801DE460
:10266700F8FE7902E559B55A08D8F9DEF7D9F5D356
:1026770022A85AE6123711055A535A4F1245C3C3B7
:102687002274FF12258CEF7001221215E340FA7AAB
:10269700017D0012264A5004DDF9DAF71226A9D285
:1026A700202274F312258C1215E340DDC082C0830B
:1026B70090E4F3E0D083D08212258C1215E32274C4
:1026C700FF1225F8EF7004C225803D1226664038B8
:1026D70012266612266674E81225F8122666740317
:1026E7001225F812266674F41225F812266674E687
:1026F7001225F812266674F31225F812266674144A
:102707001225F8122666D2252230010A12210F4718
:102717004F4F440D0A00223001FC12210F42414461
:102727000D0A002230010612210F0D0A002240086F
:1027370012210F4F4646002212210F204F4E002232
:1027470012210F2020002275A0E479E9E4F319F3A0
:102757007C10C3ED33FDEA33FA75F002A80143009C
:1027670001E235E0D4F218D5F0F7DCE675F003A8FE
:1027770001D375A0E4E230F003088001C4540F5080
:102787000D700A20F20330F10574208003C3443032
:10279700302104F0A3800E300508101E08120EF930
:1027A70080031245EAD5F0CA22301749C217547F71
:1027B700F890E4ECE0540FF94400F5827583E6E8FD
:1027C700F0E9B576028879B90400400A74404912E5
:1027D7002946E01229460212E7E854F0D2F0B42065
:1027E70002C2F07583F0E9C403F5827866C2F1127C
:1027F700380D0212E730E60990E4ECF0D217021226
:10280700E7B4160ED23F90E4F7E4F00212E7121F86
:102817004022B4010D303F05C23F122815D21D02D8
:1028270010F4B40C08121F0DC21D0212E7B40208FF
:10283700121EE3C21D0212E7B4150302190AB431CE
:10284700061218D40212E7B43007D248C21D02108C
:10285700F4B40808748012258C0212E7B40B0EA892
:1028670076B80400501874AA42C00212E7B40A14DA
:10287700A876B804005007C312416F0212E7122965
:10288700460212E7A2E792F0C2E7B419004013B478
:102897002E00500EA2F092E7F557755600D20402AB
:1028A70012E70212E7301D10540FF576C271C2709D
:1028B700C21D121DDD0212E7304811C248C218209E
:1028C700190D9039115403934529F5290212E7C0D0
:1028D700E07430122946D0E054031229460212E769
:1028E700C0E075A0F47819E230E2FCD0E0781BF282
:1028F7002275A0F47819E230E0FC781BE222122955
:10290700145003B4800122F812100180F1C310683B
:102917001DC000C0017800790A1229364006D8F98F
:10292700D9F77404D001D0003001031245EA229090
:02293700F41991
:10293900E020E003C3E42290F41BE0D322F8202333
:1029490006B4EF03D22322302403FF8016B4010218
:10295900800CB430028007F85300F0B84004D22448
:10296900FE22FE122905E41228E7EEA22392E712BD
:1029790028E7302404EF1228E7C223C22422FF09E2
:10298900FF050301020CFF0A080604462FFFFF4C4E
:1029990048FF4A7131FFFFFF7A736177324EFF6357
:1029A90078646534334FFF447666747235FFFF6E81
:1029B9006268677936FFFFFF6D6A753738FFFF4137
:1029C9006B696F3039FFFF42436C3F703AFFFFFF7D
:1029D90040FF3C3BFFFF7C49473DFF3EFFFF1B1C7F
:1029E900FFFFFFFF45FFFF11FF1417FFFFFF1060F7
:1029F900121516182E7B0B5E135D5C190EFFFFFF77
:102A0900FF077DFFFFFFFFFFFFFFFFFFFFFF617371
:102A1900646668677A786376FF627177657279743C
:102A29003132333436353B39373A38303D6F753CBE
:102A39006970476C6A406B3F3E41436E6D42464444
:102A49002F45FF2E4A4F481A4C58595756FFFF60D9
:102A5900FF5CFF5EFF7BFFFFFF5B5FFF5DFFFF9991
:102A69001011121314151617FF1819FFFFFF050689
:102A790007030809FF0BFF0DFF0EFF0AFF0CFF0FED
:102A8900505254510453025501494D4BFF28FF9EA2
:102A99009C9F9D01020A030B040C054B06A907081C
:102AA900094C560F0D0E58A0A157592E3132333407
:102AB9003536373839303A3B2F45509B5B5C28A275
:102AC90060A3524671776572747975696F703C3D80
:102AD900514D1718195DA4A553FF4A6173646667C0
:102AE900686A6B6C3F403E475F14151610A654A7E1
:102AF9007B487A786376626E6D41424349FF1112D1
:102B090013AAABAC9A7C4E444F55FF5EFF2D44B1DE
:102B1900C0B3B4B5B740B9B0B8BB413A424330319C
:102B29003233343536373839BF3FC13BC2C3B2E1DE
:102B3900E2E3E4E5E6E7E8E9EAEBECEDEEEFF0F1F4
:102B4900F2F3F4F5F6F7F8F9FA3C3E3DB6BA2F611F
:102B590062636465666768696A6B6C6D6E6F7071D4
:102B690072737475767778797ABCBEBDAF1B6030A5
:102B79003132333435363738392D3D5B5D5C3B278F
:102B89002C2E2F2008090D1B7E2921402324255E88
:102B9900262A285F2B7B7D7C3A223C3E3F20080970
:102BA9000D90E4EAE0C0E0A3E0C0E022C083C08267
:102BB90090E4EAD0E0F0A3D0E0F022BE0B0BD27093
:102BC900D215C26FC238022C6ABE0C0BD271D21553
:102BD900C26FC238022C6ABE0A22120EBFD21AC2B2
:102BE9006FC271C27090E4C5E4F0902CC4122BB589
:102BF900122D6890079A120EF4022C6ABE0D15C2A6
:102C09003EA81F12323E403A120EBF7491120F05B0
:102C1900120F2C22BE0A004005203E02804AD23EF5
:022C2900C238AF
:102C2B001231EC120EB8E51FB4CD09E577B4630091
:102C3B00500D800C500AE577B40900500280012238
:102C4B00C23E1233784007B5770280074005122C3D
:102C5B0011800CF576C270C271C238D26FD21512C8
:102C6B002DE4120EBF22C23890E4E4E576F0902CEE
:102C7B007F122BB590E4E4E0BE0D0DD26FD215F5AB
:102C8B0076902BC4122BB522BE0E0814B4FF10E5A0
:102C9B0077800CBE0F1904B5770280034001E4F076
:102CAB00AF76F57674C0120F05120F228F762212B3
:102CBB000EE0902BC4122BB52290E4C5E0F8BE0BAE
:102CCB000704B40D0CE48009BE0C1E14B4FF02748F
:102CDB000CB404028008B40C028003B40B08A95F87
:102CEB00530107B902D8F08074BE0A58105415C2AC
:102CFB001A902BC4122BB5122DE4120F1D120EE0DD
:102D0B00120EBF229007B0120EF49007C6120EF4EB
:102D1B00902D27122BB590E4C5E4F022BE0B028058
:102D2B0003BE0C1290E4C5E0F4F09007DC60039056
:102D3B0007E1120EF422BE0DFC90E4C5E070B01258
:102D4B00191080ABBE0DBCE823F8903477E893F9EB
:102D5B00A3E893F5828983122BB5022BAA90E4C5C5
:102D6B00E0F875F014A42435F582E5F03435F583DD
:102D7B007480120F057C14120F0C122D8C122D95D2
:102D8B00229034EFE893120F052290E4C5E0FC90FB
:102D9B0034AD230493C0E0EC2393C0E022900716DC
:102DAB00120EF4903639120EF490E4C5E0F890341C
:102DBB00C67C00E4A39370030C80F8ECB500F4120E
:102DCB000ECD7429120EF974D3120F05120EB81210
:102DDB002DE49031EC122BB522E490E4E3F0A3F058
:102DEB00A3F0751FCBC23E22900716120EF490363D
:102DFB0045120EF474C9120F05122D9590327512EF
:102E0B002BB522903650120EF4903679120EF4E553
:102E1B0076122FAA74C4120F05E576120F40E576D1
:102E2B00122E4D7490120F05120EB890E4C7E4F0F9
:102E3B0090E4C6E4F090E4C8E576F0902E62122B95
:102E4B00B522120F495382C075A0E779007C40E48C
:102E5B0093F3A309DCF92290E4C7E0FFBE0F080F40
:102E6B00BF110D7F008009BE0E221FBFFF027F1016
:102E7B0090E4C7EFF070097490120F05740D800782
:102E8B0024C3120F05740E90F800F022EF7036BEBB
:102E9B000B0A122F0004B50010E4800DBE0C7B1240
:102EAB002F0014B4FF03E50014F090E4C8E0FF1208
:102EBB002FAA74C4120F05EF120F407490120F0556
:102ECB00EF122E4D22BE0B0B122F0804B47E107482
:102EDB0020800CBE0C44122F0814B41F02747DF01A
:102EEB00F8120EBFE8120EF9EF24C3120F05740E81
:102EFB0090F800F022A8770890E4C8E02290E4C88C
:102F0B00E05403C4F890E4C7E014540F42007583F7
:012F1B00E7CE
:102F1C007400543F48F582E022BE0A13120EBF74AF
:102F2C0080120F057C149035AD120F0C02329DBE31
:102F3C000D1990E4C7E06013122F5890E4C7E4F029
:102F4C007490120F05740D90F800F02212084E9038
:102F5C00E4C8E0120F495382C075A0E7790012EF64
:102F6C008022903650120EF4903663120EF4E576F1
:102F7C00122FAA121517122FB7121517122FD07461
:102F8C0090120F05120EB890E4C7E4F090E4C6E47A
:102F9C00F090E4C8E576F0902FFE122BB522C0E03D
:102FAC007491120F05D0E01232D722780D540F1401
:102FBC00F5F074C3120F0512319F1231CA90E4C997
:102FCC00E5F0F022F8540FB40400400824FDF5F0AD
:102FDC007803800CE8C4540F90330793F5F0780411
:102FEC0074CA120F0512319F1231CA90E4CAE5F06F
:102FFC00F02290E4C7E0FFBE0F080FBF030D7F0067
:10300C008009BE0E3C1FBFFF027F02BF020990E485
:10301C00C9E0B4030050E090E4C7EFF0120EBF908B
:10302C003049E493600B120F05741D120EF9A38046
:10303C00F1903049EF93120F05120EB82290C2C9CD
:10304C0000BE0B0A12316104B50010E4800DBE0CF9
:10305C004B12316114B4FF03E50014A982B9C80AFC
:10306C00C0E01230C7D0E090E4C8F090E4C8E012A1
:10307C002FAA90E4C7E0700E90E4C8E07583E64494
:10308C0000F582E0800312317AC0E0122FB7D0E055
:10309C00122FD090E4C7E0FF12303D22BE0A13126B
:1030AC000EBF7480120F057C14903599120F0C0210
:1030BC00329DBE0DE690E4C7E0D25412317AFB90FB
:1030CC00E4C8E0FEB576028B797583E64400F582A0
:1030DC00EBF0EEF8F9121EA4F912218120F72D2045
:1030EC00F61BEB54F0D2F0B42002C2F07583F0EE74
:1030FC00C403F5827866C2F112380D8042E9C454DB
:10310C000F4440122946EB1229468033E9C454037C
:10311C00F8E9540F4440F930F61174EF122946E9DE
:10312C00122946EBD2E7122946801474EF1231555E
:10313C00E912315574EF123155EBD2E7123155903B
:10314C00E4C7E4F0FF12303D22C0E0E8124093D017
:10315C00E01240C422BF0107780590E4C9E0227850
:10316C000490E4CA5006A8770890E4C8E02290E4E2
:10317C00C9E090318893B444004006220102034414
:10318C0055F890E4CAE09033EA9354F0482290E466
:10319C00C5E0F89034FDE89390E4C0F090350BE86E
:1031AC009390E4C1F0903519E8230493F9E8239344
:1031BC0090E4C3F0A3E9F02290E4C2E0F5F090E4CF
:1031CC00C0E0FCC0F0A4D0F0F990E4C0E0FC90E4C6
:1031DC00C3E0F8A3E029F582E438F583120F0C2242
:1031EC00A81FBE0A00500F75A0E4EEF208B8CF136A
:1031FC001818F208800DBE0E028003BE0F5B18B8C3
:02320C00CA01F5
:10320E0008881F80007491203E0274D1120F05129F
:10321E00323E400A9007177C03120F0C8007D2052E
:10322E0012274EC2057493203E0274D3120F05224C
:10323E00B8CB02C3227E0090E4CBE0CE75F00AA498
:10324E002E500205F0FEA318B8CBEF90E4E4F0FD8B
:10325E00A3E5F0FAF0D322BE0A028033BE0D5E1251
:10326E00323E403E02346690E4C1E0F890E4C2E0A3
:10327E00BE0B0704B5000CE48009BE0C0F14B4FF9E
:10328E0002E814F074C9120F051231C4BE0A109070
:10329E00079A120EF4120EBF902CC4122BB522BE3A
:1032AE000D1B90E4C5E0F8B400028002D2549034B5
:1032BE009393E8230493C0E0E82393C0E022E4A2B2
:1032CE003892E0FC023362E5772401FDE43400FA23
:1032DE0002336EE55F540FB402057C00023362B414
:1032EE0004047C01806EB4056B7C028067E55FC4CC
:1032FE00540790330793FC805B000001030002909B
:10330E00E4FEE0FD90E4FCE0FA53020F805290E5FB
:10331E0004E0FC803F90E4FAE0FD90E4F8E0FA531C
:10332E00020F803C90E4F3E0F4541FFD7A00D21EAD
:10333E00802E90E4F3E0F4546003C4FC801690E514
:10334E0030E0FD7A00D21E801790E4F6E0FD7A00A0
:10335E00D21E800C12319A90E4C2ECF01231C422CB
:10336E00D20512274EC205C21E2290E4E5E0F5F00A
:10337E00B40200500E90E4E4E020F005600514C3A2
:10338E002260FBD32290E4C2E0A2E09238023460C5
:10339E0012337840046002F57702346090E4C2E0A4
:1033AE009033D093F9540FB40209E55F540FB40271
:1033BE0002A95F895FC00012045512047DD000027D
:1033CE00346012445590E4C2E09033EA93F55FF90D
:1033DE00895FC00012047DD0000234601222523286
:1033EE0090E4E5E090E4FCF0A3F090E4E4E090E4F7
:1033FE00FEF0A3F0805C90E4C2E090E504F0805211
:10340E0090E4E5E090E4F8F0A3F090E4E4E090E4DA
:10341E00FAF0A3F0803C90E4E4E0F4541FFC90E456
:10342E00F3E054604CF0802A90E4C2E0F45403239D
:10343E00C4FC90E4F3E0541F4CF0801690E4E4E0FA
:10344E0090E530F0800C90E4E4E090E4F6540FF058
:10345E008000122D8C122D95120EBF90079A120E0F
:10346E00F4902CC4122BB522222DF32DA82DF32D62
:10347E00F32DF32F6E2E0E2DA82DA82DA82DA82DD1
:10348E00A82DF32DF3339333EE340433AA33D33410
:10349E00763476339E344A3454340E3424343632F1
:1034AE00CC330D331C32E132FB3476347632D533E5
:1034BE004C335733233332334000312D39393900F1
:1034CE000000000000322D32353600312D3136002D
:1034DE00312D313600312D39393900322D3330004E
:1034EE00008B8C8F8A87D4D48F919191928AD4033A
:0D34FE0000030A0A000000000000000703A0
:10350B00020002030400000000000000040536DB8B
:10351B00000036D5368F36AD0000000000000000ED
:10352B0000000000000036E136FD5363616E206D34
:10353B006F64651D20202020202020202020536335
:10354B00616E2074696D651D2020202020202020B5
:10355B002020506F776572206F6E207363616E1D34
:10356B002020202020204B6579626F6172641D2022
:10357B00202020202020202020204D6F7573651DDA
:10358B0020202020202020202020202020204350DD
:10359B0055206B6579626F6172642F6D6F75736502
:1035AB002020435055206E616D6573202020202014
:1035BB002020202020204D6178696D756D20706F63
:1035CB007274731D202020202020457870616E734B
:1035DB00696F6E2077696474681D20202020457800
:1035EB0070616E73696F6E20756E6974731D202028
:1035FB002020566964656F20626C616E6B20746964
:10360B006D651D2020204B422072617465206B6517
:10361B0079732F7365631D2020204B422064656CEA
:10362B0061791D2020202020202020202020C04E2A
:10363B0065772076616C75652800C043686F6F7382
:10364B00659E9F20008043686F6F7365209E9F7FF0
:10365B007E20204350551D00C04B421D20202020B2
:10366B004D531D2020202020202020202000C04E44
:10367B00616D65202020202020202020202020206C
:10368B0020202000504320202020202020204D618E
:10369B00632020202020202053756E202020202006
:1036AB00202050532F322020202020205365724D94
:1036BB006963736F667453657250436D6F75736591
:1036CB00536572204F74686572204E6F2059657375
:1036DB004F66664F6E20536C6F772020204D6564CC
:1036EB0069756D2046617374202020466173746583
:1036FB0073745043315043325043334D61635375B0
:10370B006E751E538021751E52801C751E7380179B
:10371B00751E2A8012751E2B800D751E7080087504
:10372B001E748003751E7030010EC0E074201245AC
:10373B00EAE51E1245EAD0E02212210F535645202E
:10374B00312E390D0A00223142392D002030342F11
:10375B0031392F393620436F70797269676874205D
:10376B00313939302D3139393620526F7365204557
:10377B006C656374726F6E696373207583F01237B7
:10378B00F47583F41237F4D2F290F0007C0478666F
:10379B00C2F175A0E67900E3C45407D2F0B402027B
:1037AB00C2F012380D5382F8E5822408F58209DC49
:1037BB00E690F4007866C2F1E55F5407D2F0B402EC
:1037CB0002C2F012380D90F4087877D2F1D2F012D1
:1037DB00380D90F4107866C2F112380D90F41A740B
:1037EB0015F07582187403F02275821274C0F0758F
:0237FB00820F3B
:1037FD00E075821FE07582047470F0758214F022FA
:10380D00438202741AF0F05382F84382007413A2BB
:10381D00F092E0F07407F05382F8438201E8F05320
:10382D0082F8438202748020F1027490F074A0201B
:10383D00F10274B0F07405F022E590543C5327C3A7
:10384D00422722300112C0E074731245EA746312EC
:10385D0045EAE81245C3D0E0903AFF93FAC3123817
:10386D007D7C08E81312387DDCFAD312387DC32233
:10387D00CA858AF020F7FA858AF030F7FA400452AB
:10388D00C88004F442C8F4023DB77583F030E303F9
:10389D007583F4C4032401F582E030E21B5382F8F2
:1038AD00438203E8F030010E74721245EA746D1212
:1038BD0045EAE81245C3C322D3755D00227583F036
:1038CD00F830E3037583F4C4032401F582E020E0AE
:1038DD0003C3E4225382F8438203E0D322E8B57890
:1038ED0000401C90390D93FE55906004EE42272246
:1038FD00EE5527600AE8784D123897EEF4522722DC
:10390D000408102010204080855600755300301893
:10391D00047E02800A7583E6857682E0540FFE757B
:10392D00A0E479B0BE04028033B81A028003B89ABD
:10393D002BEE142323FE903955755300EE9360073B
:10394D00F3090E055380F5223ABA000058F05800DD
:10395D0014F014000000000077F77F00E8600AA261
:10396D00E792F03018470239F4BE03030239FD40E7
:10397D0011E557A2E792F0C2E7B4190040EEF80244
:10398D003A417457B4050050E374E0F309755301DF
:10399D00E5571423255714F8903AE3BE0103903AE6
:1039AD00D7E89360070553F3A30980F522BE0134D0
:1039BD00E8547FB40F0C30F0028035903AEF780068
:1039CD0080DF123A616009A2F092E7F3755301228C
:1039DD0090424374E0F309E8547F93A2F092E7F329
:1039ED0075530222BE0245E8547FB40F1130F00624
:1039FD00755300C20422903AF678000239AE123A9D
:103A0D0061600F75530130F00674F00553F309E84A
:103A1D00F3229042C375530274E0F30930F0097438
:103A2D00F00553F30953007FE893F322BE0305120B
:103A3D003A6180CFBE0405123A8A8003BE0514E5B3
:103A4D0056700A903AEAE8C2E7930239D4123A6105
:103A5D000239D422EE14904343C0F075F080A424B3
:103A6D0043F582E5F0D0F03443F583E8C2E793B433
:103A7D00FF07D0E0D0E00239FD6001F822B81A034B
:103A8D00D38004B89A0AC31214F892E2F0D220221D
:103A9D00B87C171214F8D220B2E2F0D2F078FC30D4
:103AAD00E207C2F0787C75530122B8FC07D0E0D054
:103ABD00E00239FDB87B071214F8B2E18008B80EA8
:103ACD00081214F8B2E0D220F0222A0000360000CD
:103ADD00AA0000B60000120000590000F01200F01C
:023AED0059007E
:103AEF00E11D45E19DC500E11477E1F014F0770089
:103AFF00FBFEEFBF51762D02040103191A31334833
:103B0F00495F61300F7374757FF9E57412409374D8
:103B1F00EF1240BBE574124093E91240BB22D273FF
:103B2F0030180280257583E6857682E0C4540775C8
:103B3F00A0E479B8B40407123B64755C0222400715
:103B4F00123B8E755C0522B40104123BEE22123C2F
:103B5F0015755C032290E4BDE0F5F0A3E0A2F492AA
:103B6F00E6D2E790E4B9F090E4BFE0A2F592E7F473
:103B7F0004A2E792E6A2F0B392E790E4B8F02290A5
:103B8F00E4BDE0F875F080F4A2E092F2A2E192F0C9
:103B9F00A2E292F1E5F090E4B8F088F0A2F490E49C
:103BAF00BEE090E4B9123BC4A2F590E4BFE090E40C
:103BBF00BA123BC422401420E7047800801B04F89B
:103BCF0053007F7002787F747F800EB480004004B2
:103BDF0078008005D2E7F87480F0A3A3E8F0227C88
:103BEF000390E4BD75A0E478B8E0F208A3DCFA75A1
:103BFF005C03227C03A85A90E4BDE6F008A35300AF
:103C0F004FDCF7885A2290E4BDE075F040A2E092B5
:103C1F00F5A2E192F4A2E492F1A2E592F390E4BE50
:103C2F00E0A2E692F0543F90E4B9F090E4BFE0A236
:103C3F00F392E7F404A2E692F2A2E792F3543F90D4
:103C4F00E4BAF090E4B8E5F0F02279387B30D25541
:103C5F00E95403C074F57412415BD0745002805F55
:103C6F00E578601DE95403F8B578005004740180BD
:103C7F002D90E530E08578F0A428C39578F5828003
:103C8F0007E954032400F5827583E6E05407B40472
:103C9F0002802C4005123CDC8025E0C45407C0E0B4
:103CAF00123DD1D0E0B4010B430104123DD15301B9
:103CBF00FB800CC2E0B40207E95403F81238EA099A
:103CCF000B309803121D71B93C86C25522E754037D
:103CDF0060028077E954031238CAFE400122300196
:103CEF00031245C3B710087700123D0A023D7FB497
:103CFF00013277037E00123D0A80507583E5E95447
:103D0F0003F84410F582EEA2E292F0A2E092F1A243
:103D1F00E392F2A2E192F3E5F0540FF0E576B500ED
:103D2F004FD22022B40E0777101241AD8042B40F4C
:103D3F000477068016B402028025B403028020B4F3
:103D4F000A02801BB40B0280168025E790423A933B
:103D5F00F8E954031238504017171241AD8011E99A
:103D6F005403B5760B90E4D02582F582EEF0D27530
:103D7F0022300112C0E074731245EA746B1245EAE7
:103D8F00E81245C3D0E0C3123DA77C08E813123DEB
:103D9F00A7DCFAD3123DA722CA858AF020F7FA854D
:103DAF008AF030F7FAB392B2858AF020F7FA858A53
:103DBF00F030F7FA858AF020F7FA858AF030F7FAB3
:103DCF00CA22E954039040B793FAE9A2E2E5C8503A
:013DDF0002E1
:103DE000E5C0FE5A7036EE035A6031E95407123FBF
:103DF000D8304A1120D005300705800B30070874F1
:103E000033C24A8002742230010CC9A2E2C94003C5
:103E1000023E131245C3304A03023E1F023F5BE7D6
:103E2000B4107F770DE920E247540390E4D0FC25DD
:103E300082F582E0B4ED1DEE7583E58C824382103D
:103E4000F0121506507CE07583E58C82438210F0F9
:103E5000D220806EB4F019EE7019ECB5780085763A
:103E60008240028C827583E6E0540323232416F7F4
:103E7000023F5BECB5780085768240028C827583C8
:103E8000E6E0540FB404005006E054F04E8003EE18
:103E90004410F0121506502A303902D251E0F5795B
:103EA00080209041F27C20B93C00400590421E7C6D
:103EB0003AA3A3ECB5820EB43A047429800F770DAF
:103EC000805C023F5BE493B506E7A3E493F7E95413
:103ED0000730E24AC2E2B57403755C00D2E2BEE983
:103EE0001B750504F500E8124093E50524088312CC
:103EF00040BBD505F1023F5B640000FA90391154D4
:103F00000393BEF4054229023F5BBEF50C2018F76F
:103F10002019F4F45229023F5BBEFFEB80EFE95415
:103F20000390E4D02582F582EEF0E95403B57414D1
:103F3000EEB4FC04D24B8023B4E0004002C24B300C
:103F40004B028017B4FF147583E5E95403F58243EF
:103F50008210E4F0E582B57402D220E75403604990
:103F60008B0006E6FEE7B4080050079041BC936E54
:103F70007037E9A2E2E5C85002E5C0035A700316A3
:103F80008027E95403C074F57412415BD074401962
:103F9000E95407124093E79041C4931240BB500389
:103FA0001680061776001241AD2290E4E7E0D5E0D6
:103FB000027406F0B4062078387E13E65E600FB215
:103FC0004020400A76005300F77600430008E528B9
:103FD00003F52808B840E222A2E2924AC0E012406B
:103FE00093D0E054039040B793C002FA7C087E005F
:103FF000124060E5C8304A02E5C05AC36001D3EE02
:1040000013FEDCEC124060E5C8304A02E5C05AC23B
:10401000076002D207124060E5C8304A02E5C05A84
:10402000C24A6002D24AC3124042E572F442C8E575
:1040300073F442C074FFF570F571F572F573D00238
:10404000EE22C0E0400AE57252C8E57352C0800A11
:10405000E572F442C8E573F442C0D0E07F0180020B
:104060007F04DFFEC0E0E57052C8E57152C07F0EEC
:10407000DFFEE570F442C8E571F442C0D26DE57030
:10408000F4600455C88005E571F455C07002C26D36
:10409000D0E022FE20550430190122A2E2C2E290B3
:1040A00040B3934006F57003F57222F57103F57382
:1040B000D26D22F7FDDF7F04011040205506301934
:1040C00003022946300130C0E0EE20E21430010E38
:0240D000C0E04E
:1040D20074201245EA74731245EAD0E00240F230CD
:1040E200010EC0E074201245EA74701245EAD0E075
:1040F200D0E01245C3C0E0EEA2E2C2E29041579383
:10410200FC7F00E5C85002E5C04C046006DFF4D332
:10411200D0E0221221C1D0E0C2A9C3124042306DC8
:1041220025A2D0B37C0913124042306D19DCF7D3BB
:10413200124042C37570FF7571FF7572FF7573FF90
:104142001221A5D2A922D3FCE572F442C8E573F488
:1041520042C0EC80DFF3FCCF3FC0E07409257483DA
:1041620055D8D36001C3D0E0220201080490417EF9
:10417200E574934004F452C02242C0220802208017
:1041820020182720192412415B401FE579B4440905
:1041920075F0FF78B61245F522B4550EE574780D28
:1041A200123850E574788D12385022E924CB8352AC
:1041B2002822FEEFFDDFFBBF7FF7000A01000001AE
:1041C200030100AAFA000000AAFA0083ABFA00FA7F
:1041D200000000FA00000000FA000001FA000002EC
:1041E200FA000003FA0000EE000000FE000000BF2B
:1041F200B0FAFF02F20BED11F311F40DF011F50D0F
:10420200F60DF70DF80DF90DFA0DFB11FC0DFD1170
:10421200EE25D229EF2F020003000A000B00FF0750
:10422200F60DF50DF40DF311F216E811E70DE60D9A
:10423200E507EA0DE900F00D007F04FF0000FE0033
:104242000000000000000000000000000000370035
:10425200000000000000000000000000000000005C
:10426200000000000000000000000000000000004C
:10427200000000000000000000000000000000003C
:104282000000000000000000000000001D00385B7C
:104292005C5253474F495148504B4D003500000086
:1042A2001C000000000000000000000000000000F0
:1042B20000000000000000000000000000000046B6
:1042C2005D000000000000000000000000007C0013
:1042D20000000000000000000000000000000000DC
:1042E20000000000000000000000000000000000CC
:1042F20000000000000000000000000000000000BC
:104302000000000000000000000000001400111F67
:104312002770716C697D7A75726B74004A000000B7
:104322005A00000000000000000000000000000031
:104332000000000000000000000000000000007EFD
:104342002F003B3C3D3E3F404142434457580046CC
:1043520000524F50514B4C4D474849FFFFFFFFFF62
:10436200FFFFFFFFFFFFFFFFFFFFFFFFFFFFFF0159
:10437200290B02030405060708090A0C0D1A1B2B58
:104382002728333435390E0F1C2A361D0038005BBE
:104392005C00000000000000000000FF00374A4EF1
:1043A20000531E302E2012212223172425263231BB
:1043B200181910131F14162F112D152C453A5400DD
:0143C200FFFB
:1043C300000506040C030B830A01097807007E002D
:1043D3007069727A6B73746C757DFF6061FFFFFFA8
:1043E300FFFFFFFFFFFFFFFFFFFFFFFFFFFF760E54
:1043F30045161E26252E363D3E464E55545B5D4CD6
:104403005241494A29660D5A1259140011001F27B7
:1044130000000000000000000000FF007C7B79002A
:10442300711C322123242B3433433B424B3A314416
:104433004D152D1B2C3C2A1D22351A77588400FF5D
:1044430000070F171F272F373F474F565E575F62EF
:10445300706972786B73746C757DFFFFFFFFFFFFEC
:10446300FFFFFFFFFFFFFFFFFFFFFFFFFFFF080E41
:1044730045161E26252E363D3E464E55545B5C4C56
:104483005241494A29660D5A1259115819398B8CD0
:1044930067646E656F6D6360616AFF777E847C79A4
:1044A300711C322123242B3433433B424B3A314496
:1044B3004D152D1B2C3C2A1D22351A7614FFFFFFA8
:1044C300007A78637660616264656D676F696B71AA
:1044D30052535455565758595B5C39377FFFFFFF8A
:1044E300FFFFFFFFFFFFFFFF7FFFFFFFFFFF3532F0
:1044F3001D1213141517161A1C191B18211E2A290D
:10450300272B2F2C313330243838367D3A7C3737FC
:104513007275737774793E3D3B3C514B434E454C2A
:1045230041000B08020E030504222628252E2D1F09
:10453300230C0F011120090D0710064739FFFF391E
:10454300000506080A0C0E10111207090B161715A1
:104553005E7071725B5C5D444546FFFFFFFFFFFFCA
:10456300FFFFFFFFFFFFFFFFFFFFFFFFFFFF1D2A0F
:10457300271E1F202122232425262829404158565F
:10458300576B6C6D792B3559636E4C0D1343787AE9
:104593002C42344A607B141B181CFF2E2F477D5A74
:1045A300324D68664F385051523D5354556A693EF7
:1045B3003F36394E3A3C6737653B646277FFFFFF0E
:1045C300300123C0E0C4540F1245E01245EAD0E0A5
:1045D300C0E0540F1245E01245EAD0E022B40A00CD
:1045E30040022407243022300107F5993099FDC297
:1045F3009922C20DD20E300112C0E0746D1245EA49
:10460300746B1245EAE81245C3D0E01248CD22D2BA
:104613000DC20E300112C0E0746D1245EA746D12C2
:1046230045EAE81245C3D0E01248CD22C20843C888
:10463300327C0FDC02804D7DFFE5C855306004DD20
:10464300F880F07C000C0000E5C8553060F7C3EC3F
:104653009467500A20082D12497BD20880D07C0031
:104663000CE5C8553070F9C3EC9409500280157DF0
:1046730008124841400E300903C38001D3E833F8E0
:10468300DDEFC322D322300A16E53352C8E5315297
:10469300C07C68DCFEE53042C0E53242C8C20A2273
:1046A30000E8B42A06D20BD20C804FC20BE854F3B5
:0346B300B4200927
:1046B600300E3EC20ED20F803AE854F3B4300930C1
:1046C6000D2FC20DD20F802BE854F3B4220A8EF0C0
:1046D6008FE0C20ED20F801B8017E8B42F0C75F046
:1046E6006375E002C20ED20F8009E8540FB40B01C5
:1046F60000C20F7C5FDCFE22124807000020F7058F
:1047060030F7070000124807800312482420F605F8
:1047160030F6070000124807800312482420F505EA
:1047260030F5070000124807800312482420F403DE
:1047360030F405124807800312482420F30530F3AD
:10474600070000124807800312482420F20530F2C1
:10475600070000124807800312482420F10530F1B3
:10476600070000124807800312482420F00530F0A5
:10477600070000124807800312482420E70530E7A7
:10478600070000124807800312482420E60530E699
:10479600070000124807800312482420E50530E58B
:1047A600070000124807800312482420E40530E47D
:1047B600070000124807800312482420E30530E36F
:1047C600070000124807800312482420E20530E261
:1047D600070000124807800312482420E10530E153
:1047E600070000124807800312482420E00530E045
:1047F60007000012480780031248240000124807E9
:1048060022C0E0E53352C8E53152C07C0EDCFEE53D
:104816003042C0E53242C87C17DCFED0E022C0E060
:10482600E53352C8E53152C07C1BDCFEE53042C0A0
:10483600E53242C87C0ADCFED0E0227CFFDC028046
:1048460023E5C8553070F67C000CE5C8553060F994
:10485600C3EC9408500AC3EC94044008C2098002D1
:10486600D209C322D32285301E85311D85321C858F
:10487600331B22851E30851D31851C32851B332254
:104886007C26DCFE8015124841C2087CFFE5C8552F
:10489600306006DCF8D2088002C208221248414085
:1048A600257D08124841300903C38001D3EE33FE4B
:1048B600DDF17D08124841300903C38001D3EF338F
:1048C600FFDDF112484122888285F0831221C1C2A0
:1048D600A912486C12495212462F402F12491A301B
:1048E6000A028002800B1246898582E08583F08069
:1048F600E61246A3200B0E300F118582E08583F069
:104906001246FE80061248861248A21248791221E3
:10491600A5D2A922200D028003200E2DE854F0B462
:1049260000028021E854F0B42010E8B42E030249B6
:104936004FE8B42A028012200D0BE854F0B4300977
:10494600200E028004D20A8002C20A22C082C083DC
:10495600E57490497393F53064FFF531E574904939
:104966007793F53264FFF533D083D08222040110A9
:10497600400C0330C07C047DC8DDFEDCFA22C2A9EF
:1049860012486C75F02C124A59124AE9124B0E2045
:104996000835124A264030D20ED279A950A7060908
:0349A60053016F4B
:1049A900A707B7FF0280040953016F89503001142A
:1049B90074201245EA744B1245EAE5061245C3E52F
:1049C900071245C31248791221A5D2A9221221C181
:1049D900C2A912486C75F03C124A59124AE9124BA5
:1049E9000E200830124A26402BD20DD279A959A798
:1049F900060953014FA7070953014F89593001147B
:104A0900744D1245EAE5061245C3E5071245C3741C
:104A1900201245EA1248791221A5D2A922124B1E69
:104A2900402D7D08124B1E4026300903C38001D357
:104A3900E50633F506DDED7D08124B1E4011300900
:104A490003C38001D3E50733F507DDED124B1E22C1
:104A590053B0CB7C92000000DCFB43B0347C1ADC01
:104A6900FE20F70530F7070000124B438003124B75
:104A79005220F60530F6070000124B438003124B13
:104A89005220F50530F5070000124B438003124B05
:104A99005220F40330F405124B438003124B522089
:104AA900F30530F3070000124B438003124B5220E9
:104AB900F20530F2070000124B438003124B5220DB
:104AC900F10530F1070000124B438003124B5220CD
:104AD900F00530F0070000124B438003124B5222BD
:104AE90053B0CB7C1FDCFE43B0347C0DDCFE20B41C
:104AF900028004C208800D7CFF20B406DCFBD208CA
:104B09008002C20822C2087C3F30B406DCFBD2080E
:104B19008002C208227CFFDC02801D20B4F97C00DF
:104B29000C30B4FCC3EC940E500AC3EC9403400857
:104B3900C2098002D209C322D32253B0CB7C0EDC36
:104B4900FE43B0347C18DCFE2253B0CB7C1CDCFE67
:104B590043B0347C0BDCFE227C26DCFE22124B4364
:104B6900000020F70530F7070000124B43800312BD
:104B79004B5220F60530F6070000124B4380031212
:104B89004B5220F50530F5070000124B4380031204
:104B99004B5220F40330F405124B438003124B525D
:104BA90020F30530F3070000124B438003124B52E8
:104BB90020F20530F2070000124B438003124B52DA
:104BC90020F10530F1070000124B438003124B52CC
:104BD90020F00530F0070000124B438003124B52BE
:104BE90020E70530E7070000124B438003124B52C0
:104BF90020E60530E6070000124B438003124B52B2
:104C090020E50530E5070000124B438003124B52A3
:104C190020E40530E4070000124B438003124B5295
:104C290020E30530E3070000124B438003124B5287
:104C390020E20530E2070000124B438003124B5279
:104C490020E10530E1070000124B438003124B526B
:104C590020E00530E0070000124B438003124B525D
:104C69000000124B43227C127DFFDDFEDCFA22128A
:104C790021C1C2A912486C75F02B124A59124AE98E
:104C8900124B6175F06275E003124B661248791296
:024C990021A553
:104C9B00D2A9224300F830E0055300FB8003430008
:104CAB000430E1055300FE800343000130E205535D
:104CBB0000FD8003430002E50022124C9E85E0823A
:104CCB007583FF1221C1C2A912486C75F02A124AD2
:104CDB0059124AE9124B618582E08583F0124B66CB
:0A4CEB00C20C124879D2A922D9495F
:104CF50002800E32FFFFFFFFFFFFFF02846175B0E8
:104D0500FF75810775E80475D8DF7590FCE4787F39
:104D1500F6D8FDE590F454C02440F57F60FEC2014D
:104D250074FFF570F571F572F573F575755060756D
:104D35005160755940755A40757B00757C0090E44B
:104D4500E77406F0755F00E57FC4FE90E5107C040E
:104D55001284C1602AFF540CD2F0B50602C2F012CB
:104D650084C120F0EBF0A3DCE77C04EFC4540FB45E
:104D7500000590E52080D9B401D690E60080D112D7
:104D850084DA12859A5389F0438901D28CD2A9D24B
:104D9500AF306B03128467E574B40400502EE579D7
:104DA5005407B4050D74382574F8E6540B601D02DC
:104DB5008373B40402801574382574F82404F9E665
:104DC50054137005E754136003028402E57BB57C38
:104DD50002802775A0E4A87CE2F9E574128DE7E965
:104DE500128E0F500A0554E554B40A09755400088B
:104DF500B810027800887C0282FD75A0F47819E26B
:104E050020E003028200781B20E534E2605BB4FFFA
:104E15001F1281C110E612A95077000953016FF7DF
:104E25000953016F89500281FBF57EC2240281D5A9
:104E3500307BD0A950F70953016F89500281FB7C63
:104E450003A9597819E230E0FC30E5E4781BE2303B
:104E55007B08129317F70953014FDCE7307BA489D0
:104E650059128956D2730281FB1281C1A2E792239E
:104E75005000F57E537E7FC224547FB40102800E1C
:104E8500B430028009F85300F0B84015D27678198D
:104E9500E230E0FC30E50302814F781BE2F57DD27C
:104EA50024202321D27C028200F208B81002780067
:104EB500227819E230E0FC20E504781BE222D0E0FC
:104EC500D0E002814F307B2875A0E4A87B74EF12F7
:104ED50081B9E57E1281B930240F307607C2767428
:104EE500EF1281B9E57D1281B9887B74801284AA9D
:104EF500107C030282FDE57EB4012FE57DFE54F0B2
:104F0500B50616E57F6E54C0700FEEF5755430C4C6
:104F1500F576D26FC2EC0282F8C27B7575FF7576A5
:104F2500FF74AA42C0C2EC0282FDB43010307B0A85
:104F3500E57D908665934529C5290282F5F85300DC
:104F4500F0B8403BF8C4657F54C07030E854033076
:104F55007B06B57403857D797583E64400F582E5A6
:104F65007DF054F0D2F0B42002C2F07583F0E8541D
:104F750003C403F5827866C2F11285610282F5B435
:104F8500091E207B030282F512844CF812844154D9
:104F95000FC44200128EAFB3E892E71284AA804D87
:104FA500B40C07307B02D2EC803BB40208C2EC742F
:104FB500AA42C08030B43117307B14E579B40400BF
:104FC500540F500BE574D2E2128DE7E4128E0FB444
:104FD5000B09307B1074AA42C0800AB40A07307BE3
:014FE50004C7
:104FE600C3128EC3307B0574801284AA306F0BE522
:104FF6005C7007E553700312848CE5537025E55009
:10500600B55103028373A851E6F5560853006F7035
:105016000686570853006F8851128669E553604229
:105026007555B075A0E4A855E2F8128EAF402FE58D
:10503600795407B4040A75F0FFE574129349801297
:105046004007E5741285A48009E574128DE7E8121D
:105056008E0F500A0554E554B40A077554000555D9
:105066001553E55C701130732F128881C273E55CAD
:105076006026755EB8C27375A0E4A95EE3F8128E69
:10508600AF406AE579C45407B4041F88F009E3F811
:105096001293664006755C00028402055DE55DB408
:1050A600104F755D00755C0080474007E5741285FA
:1050B600EB802EB40126E574908665935529602D04
:1050C6008000E574908E0B93FAE5C0035A6022E5E2
:1050D60074D2E2128DE7E8128E0F8005E574128510
:1050E600EB500A055DE55DB41007755D00055E15BC
:1050F6005C1289AD1051141020061075210280A192
:1051060012844C44901284AA0280A1128441F8535E
:1051160000070354384844C01284AA0280A175834C
:10512600E4E57444D0F582E0547F1284AA0280A19B
:105136007583E6E5744400F582E0227583E5E5743F
:105146004410F582E0540F22C3E576B50401D3225C
:10515600758C10D26B32C26B128CFE307B1C128E99
:10516600AFB3921B201C05301B108003201B0BA223
:105176001B921C74A092E01284AA22128ED6C26FD1
:10518600857674128441F579E57444FCF590D27BFA
:10519600128EAFB3921B921C22C0E075A0F4781950
:1051A600E230E2FCD0E0781BF230010312933E229B
:1051B60075A0F47819E230E0FC781BE22222222264
:1051C600225356455320312E377583F01285487584
:1051D60083F4128548D2F290F0007C047866C2F11E
:1051E60075A0E67900E3C45407D2F0B40202C2F017
:1051F6001285615382F8E5822408F58209DCE6907F
:10520600F4007866C2F1E55F5407D2F0B40202C238
:10521600F012856190F4087877D2F1D2F0128561A8
:1052260090F4107866C2F112856190F41A7415F044
:105236007582187403F02275821274C0F075820F9D
:10524600E075821FE07582047470F0758214F02296
:10525600438202741AF0F05382F84382007413A258
:10526600F092E0F07407F05382F8438201E8F053BD
:1052760082F8438202748020F1027490F074A020B8
:10528600F10274B0F07405F022E590543C5327C344
:10529600422722300112C0E0747312933E746312E7
:1052A600933EE8129317D0E090885393FAC3128581
:1052B600D17C08E8131285D1DCFAD31285D1C3223A
:1052C600CA858AF020F7FA858AF030F7FA40045248
:0152D600C80F
:1052D7008004F442C8F4028B0B7583F030E3037546
:1052E70083F4C4032401F582E030E21B5382F843C0
:1052F7008203E8F030010E747212933E746D1293BC
:105307003EE8129317C322D3755D00227583F0F828
:1053170030E3037583F4C4032401F582E020E0033E
:10532700C3E4225382F8438203E0D322E8B578002E
:10533700401C90866193FE55906004EE422722EE52
:105347005527600AE8784D1285EBEEF452272204C0
:10535700081020102040808556007553003018042F
:105367007E02800A7583E6857682E0540FFE75A07B
:10537700E479B0BE04028033B81A028003B89A2BCE
:10538700EE142323FE9086A9755300EE936007F36E
:10539700090E055380F5223ABA000058F058001458
:1053A700F014000000000077F77F00E8600AA2E72A
:1053B70092F0301847028748BE0303028751401115
:1053C700E557A2E792F0C2E7B4190040EEF802876A
:1053D700957457B4050050E374E0F309755301E57C
:1053E700571423255714F8908837BE010390882B4C
:1053F700E89360070553F3A30980F522BE0134E85B
:10540700547FB40F0C30F0028035908843780080C9
:10541700DF1287B56009A2F092E7F3755301229076
:105427008F9774E0F309E8547F93A2F092E7F3753E
:10543700530222BE0245E8547FB40F1130F00675BF
:105447005300C2042290884A78000287021287B567
:10545700600F75530130F00674F00553F309E8F354
:105467002290901775530274E0F30930F00974F035
:105477000553F30953007FE893F322BE0305128710
:10548700B580CFBE04051287DE8003BE0514E5563E
:10549700700A90883EE8C2E7930287281287B50210
:1054A700872822EE14909097C0F075F080A4249777
:1054B700F582E5F0D0F03490F583E8C2E793B4FFC6
:1054C70007D0E0D0E00287516001F822B81A03D371
:1054D7008004B89A0AC312844C92E2F0D22022B810
:1054E7007C1712844CD220B2E2F0D2F078FC30E282
:1054F70007C2F0787C75530122B8FC07D0E0D0E0F2
:10550700028751B87B0712844CB2E18008B80E08B5
:1055170012844CB2E0D220F0222A0000360000AA02
:105527000000B60000120000590000F01200F05908
:1055370000E11D45E19DC500E11477E1F014F07726
:1055470000FBFEEFBF51762D02040103191A313318
:1055570048495F61300F7374757FF9E574128DE701
:1055670074EF128E0FE574128DE7E9128E0F22D2B7
:105577007330180280257583E6857682E0C4540768
:1055870075A0E479B8B404071288B8755C022240A4
:10559700071288E2755C0522B401041289422212BF
:1055A7008969755C032290E4BDE0F5F0A3E0A2F4FD
:1055B70092E6D2E790E4B9F090E4BFE0A2F592E773
:0155C700F4EF
:1055C80004A2E792E6A2F0B392E790E4B8F0229042
:1055D800E4BDE0F875F080F4A2E092F2A2E192F066
:1055E800A2E292F1E5F090E4B8F088F0A2F490E439
:1055F800BEE090E4B9128918A2F590E4BFE090E407
:10560800BA12891822401420E7047800801B04F895
:1056180053007F7002787F747F800EB4800040044E
:1056280078008005D2E7F87480F0A3A3E8F0227C24
:105638000390E4BD75A0E478B8E0F208A3DCFA753D
:105648005C03227C03A85A90E4BDE6F008A353004B
:105658004FDCF7885A2290E4BDE075F040A2E09252
:10566800F5A2E192F4A2E492F1A2E592F390E4BEED
:10567800E0A2E692F0543F90E4B9F090E4BFE0A2D3
:10568800F392E7F404A2E692F2A2E792F3543F9071
:10569800E4BAF090E4B8E5F0F02279387B30D255DE
:1056A800E95403C074F574128EAFD0745002805F51
:1056B800E578601DE95403F8B5780050047401805A
:1056C8002D90E530E08578F0A428C39578F58280A0
:1056D80007E954032400F5827583E6E05407B4040F
:1056E80002802C4005128A308025E0C45407C0E0AF
:1056F800128B25D0E0B4010B430104128B25530112
:10570800FB800CC2E0B40207E95403F812863E0994
:105718000B3098031284D1B93C86C25522E7540352
:1057280060028077E9540312861EFE400122300190
:1057380003129317B710087700128A5E028AD3B44F
:10574800013277037E00128A5E80507583E5E95442
:1057580003F84410F582EEA2E292F0A2E092F1A2E0
:10576800E392F2A2E192F3E5F0540FF0E576B5008A
:105778004FD22022B40E077710128F018042B40F47
:105788000477068016B402028025B403028020B490
:105798000A02801BB40B0280168025E7908F8E9337
:1057A800F8E954031285A4401717128F018011E9F4
:1057B8005403B5760B90E4D02582F582EEF0D275CD
:1057C80022300112C0E0747312933E746B12933E40
:1057D800E8129317D0E0C3128AFB7C08E813128AF8
:1057E800FBDCFAD3128AFB22CA858AF020F7FA85F5
:1057F8008AF030F7FAB392B2858AF020F7FA858AF0
:10580800F030F7FA858AF020F7FA858AF030F7FA4F
:10581800CA22E95403908E0B93FAE9A2E2E5C85034
:1058280002E5C0FE5A7036EE035A6031E954071299
:105838008D2C304A1120D005300705800B30070821
:105848007433C24A8002742230010CC9A2E2C940F2
:1058580003028B67129317304A03028B73028CAFD3
:10586800E7B4107F770DE920E247540390E4D0FCB9
:105878002582F582E0B4ED1DEE7583E58C824382C6
:1058880010F0128459507CE07583E58C82438210B5
:10589800F0D220806EB4F019EE7019ECB57800855E
:1058A800768240028C827583E6E054032323241613
:0158B800F7F8
:1058B900028CAFECB5780085768240028C827583C4
:1058C900E6E0540FB404005006E054F04E8003EEB5
:1058D9004410F0128459502A303902D251E0F57936
:1058E9008020908F467C74B93C004005908F727C73
:1058F9008EA3A3ECB5820EB48E047429800F770DA4
:10590900805C028CAFE493B506E7A3E493F7E9540E
:105919000730E24AC2E2B57403755C00D2E2BEE91F
:105929001B750504F500E8128DE7E50524088312C7
:105939008E0FD505F1028CAF640000FA908665548C
:105949000393BEF4054229028CAFBEF50C2018F76B
:105959002019F4F45229028CAFBEFFEB80EFE95411
:105969000390E4D02582F582EEF0E95403B574146E
:10597900EEB4FC04D24B8023B4E0004002C24B30A9
:105989004B028017B4FF147583E5E95403F582438C
:105999008210E4F0E582B57402D220E7540360492D
:1059A9008B0006E6FEE7B408005007908F10936E4F
:1059B9007037E9A2E2E5C85002E5C0035A70031640
:1059C9008027E95403C074F574128EAFD07440195E
:1059D900E95407128DE7E7908F1893128E0F500341
:1059E900168006177600128F012290E4E7E0D5E0D1
:1059F900027406F0B4062078387E13E65E600FB2B2
:105A09004020400A76005300F77600430008E52855
:105A190003F52808B840E222A2E2924AC0E0128DBA
:105A2900E7D0E05403908E0B93C002FA7C087E0005
:105A3900128DB4E5C8304A02E5C05AC36001D3EEFD
:105A490013FEDCEC128DB4E5C8304A02E5C05AC237
:105A5900076002D207128DB4E5C8304A02E5C05A80
:105A6900C24A6002D24AC3128D96E572F442C8E571
:105A790073F442C074FFF570F571F572F573D002D5
:105A8900EE22C0E0400AE57252C8E57352C0800AAE
:105A9900E572F442C8E573F442C0D0E07F018002A8
:105AA9007F04DFFEC0E0E57052C8E57152C07F0E89
:105AB900DFFEE570F442C8E571F442C0D26DE570CD
:105AC900F4600455C88005E571F455C07002C26DD3
:105AD900D0E022FE20550430190122A2E2C2E29050
:105AE9008E07934006F57003F57222F57103F5737D
:105AF900D26D22F7FDDF7F040110402055063019D1
:105B0900030284D0300130C0E0EE20E21430010EEF
:105B1900C0E0742012933E747312933ED0E0028E5B
:105B29004630010EC0E0742012933E747012933E09
:105B3900D0E0D0E0129317C0E0EEA2E2C2E2908E6C
:105B4900AB93FC7F00E5C85002E5C04C046006DF5A
:105B5900F4D3D0E0221284CFD0E0C2A9C3128D962B
:105B6900306D25A2D0B37C0913128D96306D19DCE6
:105B7900F7D3128D96C37570FF7571FF7572FF7536
:105B890073FF1284CED2A922D3FCE572F442C8E590
:105B990073F442C0EC80DFF3FCCF3FC0E074092509
:015BA9007487
:105BAA008355D8D36001C3D0E02202010804908E45
:105BBA00D2E574934004F452C02242C02208022063
:105BCA0080201827201924128EAF401FE579B4448B
:105BDA000975F0FF78B612934922B4550EE5747828
:105BEA000D1285A4E574788D1285A422E924CB834D
:105BFA00522822FEEFFDDFFBBF7FF7000A010000FB
:105C0A0001030100AAFA000000AAFA0083ABFA0015
:105C1A00FA000000FA00000000FA000001FA000091
:105C2A0002FA000003FA0000EE000000FE00000085
:105C3A00BFB0FAFF02F20BED11F311F40DF011F5FA
:105C4A000DF60DF70DF80DF90DFA0DFB11FC0DFD12
:105C5A0011EE25D229EF2F020003000A000B00FFE4
:105C6A0007F60DF50DF40DF311F216E811E70DE63E
:105C7A000DE507EA0DE900F00D007F04FF0000FEC4
:105C8A0000000000000000000000000000000037D3
:105C9A0000000000000000000000000000000000FA
:105CAA0000000000000000000000000000000000EA
:105CBA0000000000000000000000000000000000DA
:105CCA00000000000000000000000000001D003875
:105CDA005B5C5253474F495148504B4D00350000C9
:105CEA00001C00000000000000000000000000008E
:105CFA00000000000000000000000000000000009A
:105D0A00465D000000000000000000000000007C6A
:105D1A000000000000000000000000000000000079
:105D2A000000000000000000000000000000000069
:105D3A000000000000000000000000000000000059
:105D4A000000000000000000000000000014001124
:105D5A001F2770716C697D7A75726B74004A000036
:105D6A00005A0000000000000000000000000000CF
:105D7A000000000000000000000000000000000019
:105D8A007E2F003B3C3D3E3F404142434457580032
:105D9A004600524F50514B4C4D474849FFFFFFFFB9
:105DAA00FFFFFFFFFFFFFFFFFFFFFFFFFFFFFFFFF9
:105DBA0001290B02030405060708090A0C0D1A1B20
:105DCA002B2728333435390E0F1C2A361D0038008C
:105DDA005B5C00000000000000000000FF00374A82
:105DEA004E00531E302E201221222317242526323C
:105DFA0031181910131F14162F112D152C453A544A
:105E0A0000FF000506040C030B830A01097807004A
:105E1A007E007069727A6B73746C757DFF6061FFC6
:105E2A00FFFFFFFFFFFFFFFFFFFFFFFFFFFFFFFF78
:105E3A00760E45161E26252E363D3E464E55545B99
:105E4A005D4C5241494A29660D5A125914001100F3
:105E5A001F2700000000000000000000FF007C7BFC
:105E6A007900711C322123242B3433433B424B3AB1
:105E7A0031444D152D1B2C3C2A1D22351A77588486
:105E8A0000FF00070F171F272F373F474F565E5750
:025E9A005F6245
:105E9C00706972786B73746C757DFFFFFFFFFFFF89
:105EAC00FFFFFFFFFFFFFFFFFFFFFFFFFFFF080EDE
:105EBC0045161E26252E363D3E464E55545B5C4CF3
:105ECC005241494A29660D5A1259115819398B8C6D
:105EDC0067646E656F6D6360616AFF777E847C7941
:105EEC00711C322123242B3433433B424B3A314433
:105EFC004D152D1B2C3C2A1D22351A7614FFFFFF45
:105F0C00007A78637660616264656D676F696B7146
:105F1C0052535455565758595B5C39377FFFFFFF26
:105F2C00FFFFFFFFFFFFFFFF7FFFFFFFFFFF35328C
:105F3C001D1213141517161A1C191B18211E2A29A9
:105F4C00272B2F2C313330243838367D3A7C373799
:105F5C007275737774793E3D3B3C514B434E454CC7
:105F6C0041000B08020E030504222628252E2D1FA6
:105F7C00230C0F011120090D0710064739FFFF39BB
:105F8C00000506080A0C0E10111207090B1617153E
:105F9C005E7071725B5C5D444546FFFFFFFFFFFF67
:105FAC00FFFFFFFFFFFFFFFFFFFFFFFFFFFF1D2AAC
:105FBC00271E1F20212223242526282940415856FC
:105FCC00576B6C6D792B3559636E4C0D1343787A86
:105FDC002C42344A607B141B181CFF2E2F477D5A11
:105FEC00324D68664F385051523D5354556A693E94
:105FFC003F36394E3A3C6737653B646277FFFFFFAB
:10600C00300123C0E0C4540F12933412933ED0E0FD
:10601C00C0E0540F12933412933ED0E022B40A0025
:10602C0040022407243022300107F5993099FDC233
:10603C009922C20DD20E300112C0E0746D12933E43
:10604C00746B12933EE8129317D0E012962122D271
:10605C000DC20E300112C0E0746D12933E746D12BD
:10606C00933EE8129317D0E012962122C20843C83F
:10607C00327C0FDC02804D7DFFE5C855306004DDBD
:10608C00F880F07C000C0000E5C8553060F7C3ECDC
:10609C009467500A20082D1296CFD20880D07C002D
:1060AC000CE5C8553070F9C3EC9409500280157D8D
:1060BC0008129595400E300903C38001D3E833F8DC
:1060CC00DDEFC322D322300A16E53352C8E5315234
:1060DC00C07C68DCFEE53042C0E53242C8C20A2210
:1060EC0000E8B42A06D20BD20C804FC20BE854F352
:1060FC00B42009300E3EC20ED20F803AE854F3B4ED
:10610C003009300D2FC20DD20F802BE854F3B4227E
:10611C000A8EF08FE0C20ED20F801B8017E8B42FCE
:10612C000C75F06375E002C20ED20F8009E8540FB3
:10613C00B40B0100C20F7C5FDCFE2212955B0000E9
:10614C0020F70530F707000012955B800312957855
:10615C0020F60530F607000012955B800312957847
:10616C0020F50530F507000012955B800312957839
:10617C0020F40330F40512955B800312957820F31C
:01618C00050D
:10618D0030F307000012955B800312957820F2051D
:10619D0030F207000012955B800312957820F1050F
:1061AD0030F107000012955B800312957820F00501
:1061BD0030F007000012955B800312957820E705FB
:1061CD0030E707000012955B800312957820E605F5
:1061DD0030E607000012955B800312957820E505E7
:1061ED0030E507000012955B800312957820E405D9
:1061FD0030E407000012955B800312957820E305CB
:10620D0030E307000012955B800312957820E205BC
:10621D0030E207000012955B800312957820E105AE
:10622D0030E107000012955B800312957820E005A0
:10623D0030E007000012955B800312957800001284
:10624D00955B22C0E0E53352C8E53152C07C0EDCCF
:10625D00FEE53042C0E53242C87C17DCFED0E022BC
:10626D00C0E0E53352C8E53152C07C1BDCFEE530A1
:10627D0042C0E53242C87C0ADCFED0E0227CFFDC65
:10628D00028023E5C8553070F67C000CE5C855300A
:10629D0060F9C3EC9408500AC3EC94044008C20999
:1062AD008002D209C322D32285301E85311D85324D
:1062BD001C85331B22851E30851D31851C32851BA7
:1062CD0033227C26DCFE8015129595C2087CFFE5F5
:1062DD00C855306006DCF8D2088002C2082212953B
:1062ED009540257D08129595300903C38001D3EEA5
:1062FD0033FEDDF17D08129595300903C38001D37E
:10630D00EF33FFDDF112959522888285F08312849B
:10631D00CFC2A91295C01296A6129383402F129642
:10632D006E300A028002800B1293DD8582E0858338
:10633D00F080E61293F7200B0E300F118582E08569
:10634D0083F012945280061295DA1295F61295CDBD
:10635D001284CED2A922200D028003200E2DE854E6
:10636D00F0B400028021E854F0B42010E8B42E03FC
:10637D000296A3E8B42A028012200D0BE854F0B463
:10638D003009200E028004D20A8002C20A22C08285
:10639D00C083E5749096C793F53064FFF531E574CD
:1063AD009096CB93F53264FFF533D083D0822204DF
:1063BD000110400C0330C07C047DC8DDFEDCFA22E8
:0263CD004F552A
:00000001FF
